:1000000010C02AC029C028C027C026C025C024C0CF
:1000100023C022C021C020C01FC01EC01DC01CC0E4
:100020001BC011241FBECFE5D2E0DEBFCDBF10E064
:10003000A0E6B0E0EEE8F1E003C0C89531960D927D
:10004000A036B107D1F710E0A0E6B0E001C01D92E4
:10005000A336B107E1F73BC0D3CF9FEF97BB94BB6B
:1000600080EF8ABB91BB0895F92FE82F20E030E0A4
:100070008E2F9F2F64E670E078D02817390718F488
:100080002F5F3F4FF5CF0895C89B03C082E090E0FB
:100090000895C99B03C084E090E00895CA9B03C003
:1000A00081E090E0089589B3992723E0969587959C
:1000B0002A95E1F7282F392F2170307080FF03C077
:1000C00083E090E00895932F822F08950895CFE55F
:1000D000D2E0DEBFCDBFC1DFDC9A8EE190E0C4DFAD
:1000E000DC988EE190E0C0DFDC9A81E080936200D2
:1000F00080936000C9DF282FC81759F199278230F3
:10010000910591F0833091051CF4019739F021C0DD
:100110008330910589F00497A9F01BC0809162009B
:100120008F31B8F48F5F05C080916200882389F019
:100130008150809362000DC0809160008F3148F43F
:100140008F5F05C080916000882319F081508093F3
:1001500060008091620088BB9091600095BB890F20
:100160008093610082BBC22FC5CF5527002480FF3A
:1001700002C0060E571F660F771F6115710521F02B
:0E01800096958795009799F7952F802D0895F5
:00000001FF
